:0400000014EF04F005
:0800080065EF00F000000000AC
:100010000000000000000000046ED8CF05F0E0CF23
:1000200006F00001E9CF0CF0EACF07F0E1CF08F0CD
:10003000E2CF09F0D9CF0AF0DACF0BF0F3CF12F00C
:10004000F4CF13F0FACF14F0F5CF15F0F6CF16F089
:10005000F7CF17F000C00EF001C00FF002C010F093
:1000600003C011F09DAA38EF00F09EBA27EF01F00F
:10007000A3AA3EEF00F0A4BA15EF01F00EC000F005
:100080000FC001F010C002F011C003F00CC0E9FF76
:1000900007C0EAFF078E08C0E1FF09C0E2FF0AC0FF
:1000A000D9FF0BC0DAFF12C0F3FF13C0F4FF14C076
:1000B000FAFF15C0F5FF16C0F6FF17C0F7FF045092
:1000C00006C0E0FF05C0D8FF10000001E9CF1EF018
:1000D000EACF19F0E1CF1AF0E2CF1BF0D9CF1CF034
:1000E000DACF1DF0F3CF24F0F4CF25F0FACF26F0CD
:1000F000F5CF27F0F6CF28F0F7CF29F000C020F099
:1001000001C021F002C022F003C023F09DA28CEFB9
:1001100000F09EB2AEEF00F020C000F021C001F070
:1001200022C002F023C003F01EC0E9FF19C0EAFF9D
:10013000198E1AC0E1FF1BC0E2FF1CC0D9FF1DC011
:10014000DAFF24C0F3FF25C0F4FF26C0FAFF27C062
:10015000F5FF28C0F6FF29C0F7FF110002016E2B42
:100160006E51640804E16E6B010148890201A1A18E
:100170000CD00101493D05D04A3D03D0020105D014
:100180000101492BD8B44A2B02019380A19381B07D
:10019000A183A1B320D06FA11ED0362AD8B4372AAC
:1001A0006FA311D0A1914AC133F049C132F033504D
:1001B000355C08E303E13450325C04E233C035F0CF
:1001C00032C034F06F936FB306D001014A6B496BB4
:1001D0000201A1816F836F91A1B36F81010148A3D7
:1001E00014D0489333C039F032C038F035C03BF0FA
:1001F00034C03AF037C03DF036C03CF0336A326A62
:1002000035683468376A366A48859E9200018CEFFB
:1002100000F0A4AAFED79CCF31F0AACF01F031A202
:1002200002D09C989C8816EF01F0F3D701C09DF294
:10023000A49A3EEF00F09EAAFED7ACCF31F0AFCF2C
:1002400001F031A202D0AC98AC8828EF01F0F3D7CE
:1002500001C09DF202019D510D0818E09D510A0850
:1002600015E07651FB0812E3036A76514D0FE96EF3
:10027000010E0320EA6E9DC2EFFF762B036A7651D2
:100280004D0FE96E010E0320EA6EEF6A6FB524D0C0
:1002900071C270F272C271F273C272F274C273F2FE
:1002A00075C274F29DC275F27051240814E1715147
:1002B000470811E1725150080EE1735147080BE1F4
:1002C0007451470808E17551410805E1010148836F
:1002D000486A02016F8531D09D510D0803E09D51A0
:1002E0000A082BE19D6B76519D5D19E2490E9D2513
:1002F000016E036AD8B0032A03C09FF2036A9D51BE
:100300004D0FE96E010E0320EA6EEFCFA0F29FC2FF
:10031000EAFF01C0E9FFA0C2EFFF9D2BE4D7490E21
:100320009D25E96EEA6AD8B0EA2AEF6A76C247F1FB
:100330000101488702016F95766B9E9A00013EEF9E
:1003400000F0020EEA6E7B0EE96EEF5011E00A0E2D
:10035000016EBF0E006E0400002EFDD7012EF9D7EE
:100360005E0E006E002EFED700D00400EF2EEFD7F9
:100370001200C150C00B0309C16EC18EC280C18C76
:10038000C282C2B2FED7C19CF80E0F01486FC28C68
:10039000C29E4951E00B1F09496FF80E486F7F0E4E
:1003A000496F000E0609CA6E310ECB6E0E0E0201A9
:1003B0007B6F0001C6DF0101489348954897489933
:1003C000336A326A35683468376A366A4D6B0201BF
:1003D0004B6B4868496A0101476B456A446A476844
:1003E000000178EF04F0D8B204D0020EEA6E950E48
:1003F000E96E006A016A026A036A0201956B966BF4
:10040000976B986B94519311921191112CE0200EDF
:10041000996FD8908D378E378F37903795379637BD
:10042000973798379451985D08E19351975D05E1AE
:100430009251965D02E19151955D0FE39151955F67
:100440009251D8A0923D965F9351D8A0933D975F6B
:100450009451D8A0943D985FD8800036013602367A
:100460000336992FD6D795C2EFFF96C2ECFF97C2FD
:10047000ECFF98C2ECFF000192EF02F0D89002016D
:100480006C35036A4C0FE96E020E0320EA6E7EC2E1
:10049000ECFFED527DC2EFFF6C2B6C510F0801E2B7
:1004A0006C6B6D510F0801E36D2B866B856B846B54
:1004B000836B876B6D51875D14E2D8908735036A33
:1004C0004C0FE96E020E0320EA6EECCF03F0ED5202
:1004D000EF50832703508423000E85238623872B28
:1004E000E9D7D8906D31006E016A026A036A005044
:1004F0008325896F015084218A6F025085218B6F7B
:10050000035086218C6FD892906F8BC28FF28AC273
:100510008EF289C28DF2946B936B926B6DC291F2E5
:10052000000161D703C082F202C081F201C080F2F3
:1005300000C07FF202017FC201F080C202F0000120
:100540001200000E016EC250C30B0110C26E010EEC
:1005500002017B6F0001F5DE0201786B78510F0814
:1005600018E3C282C2B2FED7C4CF02F0C3CF01F0FB
:10057000C4CF7CF2C3CF7BF2C4CF7EF2C3CF7DF277
:1005800000017CDF02C07AF201C079F20201782B0F
:10059000E5D77AC23FF079C23EF0040E016EC25038
:1005A000C30B0110C26E010E7B6F0001CADE020197
:1005B000786B78510F0818E3C282C2B2FED7C4CF5D
:1005C00002F0C3CF01F0C4CF7CF2C3CF7BF2C4CF23
:1005D0007EF2C3CF7DF2000151DF02C07AF201C08A
:1005E00079F20201782BE5D77AC243F079C242F062
:1005F000080E016EC250C30B0110C26E010E7B6F5C
:1006000000019FDE0201786B78510F0818E3C28267
:10061000C2B2FED7C4CF02F0C3CF01F0C4CF7CF288
:10062000C3CF7BF2C4CF7EF2C3CF7DF2000126DFC1
:1006300002C07AF201C079F20201782BE5D77AC2C2
:1006400041F079C240F000018BEF04F002019951B2
:100650009907000A24E098C2EAFF9751972BD8B473
:10066000982BE96EEF50951B9A6B9A51070816E389
:100670009551010B006E036A005003100AE0D890F8
:1006800096319C6F9531010A956F9C51A00A966F27
:1006900003D0D890963395339A2BE7D7D8D795C205
:1006A00001F096C202F000011200A4A8FED7A96EC4
:1006B0001200180E01014725020F0201906F916B85
:1006C000D8B0912B230E786F520E796F040E7A6F8B
:1006D0000C0E7B6F7C69260E7D6F91C27EF290C2FC
:1006E0007FF245C080F244C081F239C082F238C046
:1006F00083F23BC084F23AC085F23DC086F23CC032
:1007000087F23FC088F23EC089F241C08AF240C001
:100710008BF243C08CF242C08DF246C08EF248C0CC
:100720008FF296699569020E986F790E976F170E82
:10073000996F00018BDF02C093F201C092F293C265
:1007400096F292C295F20201986B490E976F47C1DB
:1007500099F200017BDF02C093F201C092F2020124
:10076000946B945117080FE3036A9451780FE96E64
:10077000020E0320EA6EEFCF95F29551000195DF4E
:100780000201942BEED7946B010147510201945D55
:100790000EE2490E9425E96EEA6AD8B0EA2AEFCF54
:1007A00095F29551000181DF0201942BEDD793C2A0
:1007B00095F29551000179DF92C295F202019551AF
:1007C000000173DF442AD8B4452A96EF04F047525B
:1007D00004E0473C01D001D04706483C01D001D09D
:1007E000482A463C01D001D0462A3C5202E13D5203
:1007F00003E0939A8A8A02D0939A8A9A4150020817
:1008000005E2FF0A0AE140500E0807E341500308E1
:1008100007E303E14050010803E393968A8602D080
:1008200093968A969EEF04F0F86A9F829F9AA59A03
:10083000D08E078E0E01550EA76EAA0EA76EFF91E1
:100840000C0EF66F050ED16F550EA76EAA0EA76E91
:10085000FF81400E9B6ED36AD350316A7E86A00E14
:10086000B06E010E7F6EA60EAD6E900EAC6E7C86E5
:100870008A0EAB6E000E7D6EA60EA86E900E9C6E5C
:10088000FF0E0F01486FC29CC29E4951E00B1F0929
:10089000496F070EB46E02016F916F936F9507D089
:1008A00002002B000023424C000742700000000EA3
:1008B000F86E080EF76EA00EF66E0900F550006E89
:1008C000000A13E00900F550016EE8BE05D03F0BA9
:1008D000EA6E0900F5CFE9FF01BC090001AC09008F
:1008E000F5CFEEFF004EE9D7F9D7F86A000141D500
:1008F000939A8A9A93988A9893968A969D829D8ACB
:10090000C00EF2120201776B0400010148A504D069
:100910004895000116D6010148A704D0489793983E
:100920008A78476A475205E10001C3D6466A47689C
:10093000010148A904D04899000149D701010201E9
:04094000E3D7FFD723
:083FF80000F41DFFFFF9CFF1F9
:00000001FF
